:1000000012C02CC02BC02AC0CCC428C027C026C018
:1000100025C024C023C022C021C020C01FC01EC0D4
:100020001DC01CC01BC011241FBECFE5D4E0DEBF25
:10003000CDBF10E0A0E6B0E0E6E2FFE002C0059030
:100040000D92AA36B107D9F711E0AAE6B0E001C0D7
:100050001D92AE37B107E1F75AD463C7D1CFAC01D7
:100060008091B400873219F481E08093B3008091CD
:10007000B400882351F487EB90E09093B60080930E
:10008000B50087E28093B4000EC08091B400815027
:100090008093B4008091B5009091B6000296909341
:1000A000B6008093B500E091B500F091B6005183A1
:1000B00040838091B300882309F1A0E020E030E084
:1000C00067EB70E0B1E0FB01E20FF31F80819181EB
:1000D000841B950B8F3C910544F480819181FA013A
:1000E000E81BF90BE836F1050CF0AB2F2E5F3F4F04
:1000F0002035310541F78A2FA11181E00895CF9372
:10010000DF93EC01ACDF882351F48CE0CC33D807CB
:1001100030F480E0C855D44018F081E001C080E0A0
:10012000DF91CF9108959C018BE02D36380788F43C
:100130001092B200E2E3F0E08081886080838081E9
:100140008F7E8083662329F4E8E3F0E08081806479
:1001500080838BE0253D380790F082E08093B200E9
:10016000E2E3F0E08081877F80838081806180830B
:10017000662329F4E8E3F0E08081806480838CE0EA
:100180002C33380790F081E08093B200E2E3F0E096
:100190008081877F8083808180618083662329F4CA
:1001A000E8E3F0E08081806480832F5B344078F462
:1001B000662329F4E8E3F0E080818F7B8083E2E32B
:1001C000F0E080818061808380818860808380917D
:1001D000B2000895DF92EF92FF920F931F93FC01FC
:1001E000D62E4817590768F4662329F4E8E3F0E0AF
:1001F000808180648083E2E3F0E080818F7E808371
:1002000032C08091AF00882321F081508093AF00ED
:1002100003C084E18093AF00BF01621B730B80E0D9
:1002200090E066D5A8019701CDD536D52091AF00D5
:10023000621768F4DD2029F4E8E3F0E080818F7B29
:100240008083E2E3F0E08081806180830CC0DD2068
:1002500029F4E8E3F0E0808180648083E2E3F0E069
:1002600080818F7E80831F910F91FF90EF90DF90B0
:100270000895EF92FF920F931F938C01F62E81EC5D
:1002800095E0841B950B0817190710F41092B00025
:1002900089E096E0841B950B8017910740F481E07C
:1002A0008093B000E2E3F0E08081877F808382EA80
:1002B00095E0841B950B0817190728F4E2E3F0E09A
:1002C000808188608083B80180E090E011D524EAC5
:1002D00033EF47E954E472D5181694F4C8016F2D32
:1002E00048EE54E02FEB34E00F2EFFE0EF2EF0E865
:1002F000FF2EF8EF0F2FFEE31F2FF02D6BDF0CC04A
:10030000FF2029F4E8E3F0E080818F7B8083E2E343
:10031000F0E08081806180838091B0001F910F9117
:10032000FF90EF900895EF92FF920F931F938C012F
:10033000F62E9A01220F331F8DE69BE0821B930B52
:100340000817190710F41092B10089EE9BE0821B88
:10035000930B8017910740F481E08093B100E2E3B2
:10036000F0E08081877F808382EA95E0841B950B93
:10037000880F991F0817190728F4E2E3F0E080813D
:1003800088608083B80180E090E0B2D42BEF39EA36
:1003900046E155E413D5181694F4C8016F2D41EDCC
:1003A00059E02AE639E00F2EFCECEF2EFCECFF2E94
:1003B000F6E40F2FFEE31F2FF02D0CDF0CC0FF2003
:1003C00029F4E8E3F0E080818F7B8083E2E3F0E0D2
:1003D0008081806180838091B1001F910F91FF9097
:1003E000EF900895EF92FF921F93CF93DF93162F14
:1003F0007A01A0E0B0E0BC01CD017AD42DEF39E55F
:100400004EEC50E4DFD448D4DC01CB01EC0177DEC4
:10041000882391F088E0CD30D80738F0CE01612FE5
:10042000A70181DF809307010CC0CE01612FA701D6
:1004300020DF8093070105C0CE01612F74DE809319
:10044000070180910701DF91CF911F91FF90EF90FD
:1004500008959C0180916E00882351F48DE1809372
:100460006E0083E790E09093700080936F000EC061
:1004700080916E00815080936E0080916F0090910A
:10048000700002969093700080936F00E0916F006F
:10049000F09170003183208340E050E020E030E0B4
:1004A00063E770E0FB01E20FF31F80819181481741
:1004B000590714F4408151812E5F3F4F2C33310591
:1004C00089F78FEA90E09093720080937100CA01DF
:1004D00005978D33910514F08CE390E09C019923EE
:1004E00014F420E030E08CE3821B0895662331F0A1
:1004F000E8E3F0E08081806880830895AADF80933C
:100500006000809160008C3331F4E8E3F0E080819A
:1005100080688083089580916C008823C9F480915D
:100520006B00882341F0E8E3F0E080818F778083DF
:1005300010926B0008C0E8E3F0E08081806880835F
:1005400081E080936B008091600080936C0005C017
:1005500080916C00815080936C0080916C00409180
:10056000600020916D0090E0840F911D30E028170D
:10057000390754F480916C009091600020916D00D7
:10058000980F921B90936C008091600080936D0097
:1005900080916C0080916C008D3318F08CE3809317
:1005A0006C00089580916A00882389F4B69B06C088
:1005B000E8E3F0E080818F7B808305C0E8E3F0E032
:1005C00080818064808384E180936A0008958150F3
:1005D00080936A000895282F392FECE3F0E08081A2
:1005E00081FDFDCF822F932F9FBB8EBBE09A8DB3F1
:1005F0000895282F392FECE3F0E0808181FDFDCFB5
:10060000822F932F9FBB8EBB6DBB0FB6F894E29ADF
:10061000E19A0FBE0895DF93CF9300D000D0CDB7FD
:10062000DEB7AC01662309F0C6C0863991050CF02F
:10063000C2C0009709F4BFC080910D0190910E01D6
:100640009A01281B390B3A83298350930E0140935A
:100650000D01809163009091640020910B01309115
:100660000C01821B930B9C838B8380916300909180
:10067000640090930C0180930B018B819C81181670
:1006800019062CF489819A811816190644F08B8179
:100690009C81992304F589819A819923E4F484E06B
:1006A00090E0909362008093610080910A0188231A
:1006B00019F084E08093080181E080930901109291
:1006C0000A0180910801882331F082E090E0909344
:1006D0006200809361008B819C8199232CF4898135
:1006E0009A81181619064CF08B819C8118161906F0
:1006F00004F589819A819923E4F48CEF9FEF90931C
:1007000062008093610080910901882319F084E0E0
:100710008093080181E080930A0110920901809181
:100720000801882331F08EEF9FEF90936200809351
:10073000610080910801882329F08091080181508F
:100740008093080180916300909164002091610082
:1007500030916200280F391F3093640020936300AA
:1007600080916300909164008B3F910564F08AEF63
:1007700090E090936400809363008CEF9FEF9093E0
:1007800062008093610080916300909164004497BF
:1007900064F484E190E0909364008093630084E0CB
:1007A00090E090936200809361008091630090914B
:1007B00064009BBD8ABD6230B1F48091630090916A
:1007C0006400CE9764F08091630090916400992357
:1007D0000CF40196959587959BBD8ABD06C08EE168
:1007E00090E09BBD8ABD613019F0463951059CF0FF
:1007F0004837510564F084E190E090936400809361
:10080000630084E090E090936200809361008EE149
:1008100090E09BBD8ABD0F900F900F900F90CF91ED
:10082000DF91089582990FC0ECE3F0E0808181FDB3
:10083000FDCF80E090E09FBB8EBB1DBA0FB6F89451
:10084000E29AE19A0FBEECE3F0E0808181FDFDCFFA
:1008500080E090E09FBB8EBBE09A8DB380937D01DA
:1008600081E090E06BEE72E0ECD10895A7E3B0E098
:100870008C9182608C93E1E3F0E0808188608083DA
:100880008081806180838C9180648C938C9180685E
:100890008C93E5E3F0E080818860808380818061D3
:1008A0008083E2E3F0E080818460808380E888B91F
:1008B00081E88FBD89E08EBD8FE090E09BBD8ABD51
:1008C00087E085BDE6E2F0E085EC808384E487B9CB
:1008D000808180648083808186FDFDCF84B185B175
:1008E0002EE088E190E00FB6F894A89581BD0FBE88
:1008F00021BD80E489BF96DF90937C0180937B01CA
:10090000E5E5F0E080818068808378940895AEDF2B
:10091000E5E5F0E0A89580818068808388958081F6
:100920008F778083F7CFCF93DF939C0180910F0166
:10093000909110012817390769F5C90133230CF488
:100940004F969595879595958795959587959595C6
:10095000879595958795EC012A9681E090E0BE01F8
:1009600049EF52E084D1ECE3F0E0808181FDFDCFDE
:1009700080E090E09FBB8EBB8AEA8DBB0FB6F894F7
:10098000E29AE19A0FBE80937D01D0937C01C093DF
:100990007B0104C03093100120930F01DF91CF91B0
:1009A000089578941F920F920FB60F9211242F93EF
:1009B0003F934F935F936F937F938F939F93AF93E7
:1009C000BF93EF93FF93DF93CF9300D000D000D07D
:1009D000CDB7DEB7A895E6E2F0E08081806880833D
:1009E00082E487B9808180648083808186FDFDCF29
:1009F00084B1898385B18A832A813981922F80E0ED
:100A0000830F911D9E838D838D819E81899714F024
:100A10001C8202C081E08C8381E487B9E6E2F0E0C9
:100A2000808180648083808186FDFDCF84B189834D
:100A300085B18A834A8129818D819E8130E0281B7E
:100A4000390B942F80E0280F391F3E832D8340916E
:100A50001101509112018D819E81209111013091DF
:100A60001201480F591F332314F42F5F3F4FC90160
:100A7000959587959A01281B390B30931201209385
:100A80001101809111019091120199230CF40196AA
:100A9000959587959E838D838D819E81409167007A
:100AA00050916800609115019DDC8B8386E487B9C5
:100AB000E6E2F0E0808180648083808186FDFDCF66
:100AC00084B1898385B18A836A8189812091650097
:100AD000309166004091650050916600280F311DED
:100AE000962F80E0280F391F552314F4415E5F4F85
:100AF000CA0195958795959587959595879595952F
:100B0000879595958795A901481B590B50936600C9
:100B100040936500809165009091660099230CF4E4
:100B20004F969595879595958795959587959595E4
:100B3000879595958795909368008093670020919D
:100B400067003091680080917B0190917C01821B4D
:100B5000930B0AF40196959587959093680080937E
:100B6000670080916700909168000D9724F081E004
:100B70008093150102C01092150180916700909139
:100B8000680088539F4F1CF481E08093150180E436
:100B900087B9E6E2F0E0808180648083808186FD11
:100BA000FDCF84B1898385B18A83E6E2F0E080815C
:100BB0008F7780832A813981922F80E0830F911D66
:100BC00090931401809313018C81882341F081E07C
:100BD0008B838DE790E090931401809313018091B3
:100BE0001301909114016B8116DD80911301909196
:100BF00014016C814B817ADC809115018111D2DC6A
:100C000080917D018A3A29F080916500909166007B
:100C10008ADE2696F894DEBF7894CDBFCF91DF911F
:100C2000FF91EF91BF91AF919F918F917F916F91C4
:100C30005F914F913F912F910F900FBE0F901F909A
:100C40001895DF92EF92FF920F931F937B018C0117
:100C5000FB010995D82EC8010196F7010995982F37
:100C60008D2D1F910F91FF90EF90DF900895DF92EF
:100C7000EF92FF920F931F93D72E7A018C01FA0106
:100C80000995C80101966D2DF70109951F910F91E6
:100C9000FF90EF90DF90089570D088F09F5790F00C
:100CA000B92F9927B751A0F0D1F0660F771F881F91
:100CB000991F1AF0BA95C9F712C0B13081F077D0F8
:100CC000B1E0089574C0672F782F8827B85F39F096
:100CD000B93FCCF3869577956795B395D9F73EF4F0
:100CE00090958095709561957F4F8F4F9F4F089598
:100CF000E89409C097FB3EF49095809570956195B6
:100D00007F4F8F4F9F4F9923A9F0F92F96E9BB276B
:100D10009395F695879577956795B795F111F8CFE7
:100D2000FAF4BB0F11F460FF1BC06F5F7F4F8F4F52
:100D30009F4F16C0882311F096E911C0772321F048
:100D40009EE8872F762F05C0662371F096E8862FE0
:100D500070E060E02AF09A95660F771F881FDAF737
:100D6000880F9695879597F9089557FD9058440FE9
:100D7000551F59F05F3F71F04795880F97FB991FFA
:100D800061F09F3F79F087950895121613061406B7
:100D9000551FF2CF4695F1DF08C016161706180644
:100DA000991FF1CF86957105610508940895E8941F
:100DB000BB2766277727CB0197F9089566D008F4FB
:100DC0008FEF08950BD09CC08DD028F092D018F0F2
:100DD000952309F07EC083C01124EACFC6DFA0F3BB
:100DE000959FD1F3950F50E0551F629FF001729FC0
:100DF000BB27F00DB11D639FAA27F00DB11DAA1FDF
:100E0000649F6627B00DA11D661F829F2227B00D2B
:100E1000A11D621F739FB00DA11D621F839FA00DB6
:100E2000611D221F749F3327A00D611D231F849F06
:100E3000600D211D822F762F6A2F11249F5750405D
:100E40008AF0E1F088234AF0EE0FFF1FBB1F661FF8
:100E5000771F881F91505040A9F79E3F510570F0B1
:100E600038C0A6CF5F3FECF3983EDCF386957795CC
:100E70006795B795F795E7959F5FC1F7FE2B880FAC
:100E8000911D9695879597F90895990F0008550F2C
:100E9000AA0BE0E8FEEF16161706E807F907C0F000
:100EA00012161306E407F50798F0621B730B840B08
:100EB000950B39F40A2661F0232B242B252B21F4E2
:100EC00008950A2609F4A140A6958FEF811D811D82
:100ED000089597F99F6780E870E060E008959FEFBC
:100EE00080EC089500240A941616170618060906C1
:100EF000089500240A941216130614060506089590
:100F0000092E0394000C11F4882352F0BB0F40F417
:100F1000BF2B11F460FF04C06F5F7F4F8F4F9F4F57
:060F20000895F894FFCFD4
:0A0F26003C04003200CC100A000069
:00000001FF
